:1036AD0000640014000900320032000A0005000A0F
:0236BD00753066
:10311700C10B4100B30101B7010154000147000190
:103127005800015900014500014900014A00C10A40
:10313700C1000143FF41006B0041009000015C00AA
:0E314700C103C182C108014800015B00C10143
:1016EF00E4F523F5A012100090006B7403F012368E
:1016FF0008123452AF431235A3300926C209786756
:10170F00E6600B16E6B401062005031234F4E56219
:10171F00D39400400DD5620A1236F27F0A7E001272
:10172F0036E7789CE6D394034050E4F6120FFC1290
:10173F002A8BE4F55AE55A25E024A5F8E6FE08E6DB
:10174F00FF9000B4EEF0A3EFF04E6025E024FFF021
:10175F009000B4E034FFF0E0FEA3E0FFE55A25E08F
:10176F0024A5F8A60608A607EF4E7005AF5A123645
:10177F009B055AE55AC3940940BBE5547002E10832
:10178F001554744B2554F8E614601C14602614602D
:10179F003724FC603D146049240870DEB204E4FD78
:1017AF00FCFF12348C80D312028CE4FDFC7F0112FB
:1017BF00348C80C6E51C7003123452122BC1E4FD29
:1017CF00FC7F0212348C80B2E4FDFC7F0312348C58
:1017DF0080A8E4FF121800E4FDFC7F0712348C8010
:0E17EF00991221D1E4FDFC7F0812348C808C0D
:101000001236BF9000B6741EF0E4900108F0900113
:1010100008E0FFC39408501DEF25E025E024B8F553
:1010200082E43400F583120AF10000000090010808
:10103000E004F080D97B017A01790AE4F5317F156B
:10104000121F30500201FE7B017A01790AE4F5316A
:101050007F16121F304052E490010AF0A3F0900175
:1010600008F0900108E0FFC3941040022151EF24E2
:1010700015FF90010AE0FCA3E0FDE4FB1231F990BA
:101080000108E025E0FFE433FE74002FF5827400D0
:101090003EF583E4F074012FF58274003EF583E49D
:1010A000F0900108E004F080B9E4900108F09001AC
:1010B00008E0FFC3941040022151EF2415FF7B018B
:1010C0007A01790AE4F531121F3090010AE0FD90AF
:1010D0000108E025E0FFE433FE74002FF582740080
:1010E0003EF583EDF090010BE0FD74012FF5827465
:1010F000003EF583EDF0900108E004F080B0E4904C
:101100000108F0900108E0FFC394105044EF24154B
:10111000FF7B017A01790AE4F531121F3090010A50
:10112000E0FD900108E025E0FFE433FE74002FF5B8
:101130008274003EF583EDF090010BE0FD74012F09
:10114000F58274003EF583EDF0900108E004F08034
:10115000B2E4900108F0900108E0FFC3942050141D
:10116000744A2FF582E43400F583E4F0900108E03E
:1011700004F080E29001087410F0900108E0FFC3D1
:1011800094385033E490010AF0A3F0EF2415FF7B6C
:10119000017A01790AE4F531121F3090010BE0FF6A
:1011A000900108E02410F582E43400F583EFF0901C
:1011B0000108E004F080C37B017A01790AE4F5318B
:1011C0007F4D121F3040057543FF800690010BE0F4
:1011D000F543300012D2A0D2A1D2A2D2A3D2A4D27F
:1011E000A5D2A6D2A78010C2A0C2A1C2A2C2A3C289
:1011F000A4C2A5C2A6C2A7D2B4D294D295C2B7C285
:10120000B5C2B6C293C2D9C2B37B017A017909E4EF
:10121000F5327F0F12300040069001097401F09002
:101220000109E0B4010B7587809000497403F080D8
:1012300009E4F5879000497406F07580FF759850B1
:10124000758921758DFD758BFD758A04758CF7D2B6
:101250008ED28CD2A943BF02123257D2AFD2AC7514
:101260004601120FFC1236E3120FFC1236E3120F86
:10127000FC1236E3120FFC1236E3120FFC1236E3B7
:10128000120FFCE4F546900108F0900108E0FFC35E
:1012900094125018EF25E0246CF582E43400F583B5
:1012A000E4F0A3F0900108E004F080DEE49001088F
:1012B000F0900108E0FFC39408500B749D2FF8E4F0
:1012C000F6E004F080EBE4900108F0900108E0FF04
:1012D000C39409500FEF25E024A5F8E4F608F6E0E2
:1012E00004F080E7E4FBFDFC7F631231F9E4900039
:1012F0006AF07B017A0079B1F5327F0D123000403F
:10130000069000B17480F07B017A0079B3E4F53285
:101310007F0C123000400AE4FB7D01FC7F0C12318F
:10132000F99000B3E0700FFB7D01FC7F0C1231F9E6
:101330009000B37401F0E4FB7D12FC7F051231F9DB
:10134000E4FB7D14FC7F071231F97B017A00796B95
:10135000E4F5327F08123000E4FDFCFF12348CE427
:10136000FDFC7F0212348CE4FDFC7F0112348CE41E
:10137000FDFC7F0712348C9000B3E06402703BFDEB
:10138000FC7F0412348CE4900108F0900108E0FF27
:10139000C394105018EF25E02491F582E43400F551
:1013A00083E4F0A3F0900108E004F080DE90006A8E
:1013B000E030E704D2068002C206E4FDFC7F08129A
:1013C000348CE4900108F0900108E0FFC3942050B1
:1013D0001474D82FF582E43400F583E4F09001080A
:0513E000E004F080E2D2
:0113E50022E5
:03000B00022FAA17
:102FAA00C0E0C0F0C083C082C0D075D000C000C0ED
:102FBA0001C002C003C004C005C006C007758A0468
:102FCA00758CF7789C06D20978B706E6D394034045
:102FDA000276011232B1D007D006D005D004D00350
:102FEA00D002D001D000D0D0D082D083D0F0D0E0AF
:012FFA0032A4
:10369B00E554C39409500AAE540554744B2EF8A646
:0236AB000722F4
:10348C008C2E8D2FE52F452E701FEF25E024ADF5EA
:10349C0082E43436F583E493FC740193FDEF25E06C
:1034AC0024A5F8A60408A60522EF25E024A5F8A675
:0534BC002E08A62F22DE
:1036080090006BE0FF7006439B4075A303EFC394E3
:0E361800014002D20AEFC394034002D2002206
:102BC100200A02D2B3E51CB40109D20C7F08122CF1
:102BD100CE8012E51CB40205120F438008E51CB437
:102BE1000303122DAD20080281CD300A67E4F524DC
:102BF100E52425E0246CF582E43400F583E0FEA3AE
:102C0100E0FFD39464EE94005019E52425E0247C80
:102C1100F582E43400F583E0FCA3E0D39464EC9402
:102C2100004022C3EF9484EE9403401FE52425E085
:102C3100247CF582E43400F583E0FEA3E0C39484B0
:102C4100EE94034006900090E004F00524E524B4DE
:102C5100089E8068E4F524E52425E0247CF582E4DF
:102C61003400F583E0FEA3E0FFE52425E0246CF5C4
:102C710082E43400F583E0FCA3E0C39FFFEC9EFEF9
:102C81001236D1D3EF9432EE6480948040259000C7
:102C910090E004F074079524FFE55CA80708800321
:102CA100A2E713D8FB4401FEA807088002C333D86A
:102CB100FCF55C0524E524C39408409B900090E05A
:0C2CC100B4FF05C202C20822D202C20801
:012CCD0022E4
:021800008F2433
:10180200E4F528D20FE52414604A046002019985A8
:101812008027A2B7920CA2B5920DA2B6920EC2B7C1
:10182200C2B5C2B67580FFC2B47F0A7E001236E727
:10183200C294858025D2947580FFC295858026D278
:1018420095D2B4852780A20C92B7A20D92B5A20EB2
:1018520092B68043858027A2B7920CA2B5920DA2C0
:10186200B6920EC2B7C2B5C2B67580FFC2107F056E
:101872007E001236E7C212858025D2127580FFC221
:1018820011858026D211D210852780A20C92B7A290
:101892000D92B5A20E92B67D01E4FCE5255D7003C2
:1018A200D38001C3500AE5265D70028001C3400364
:1018B200ED4228ED25E0FD0CBC08E074592524F822
:1018C200E665286023744A2524F806744A2524F81C
:1018D200E6C3940A401974592524F8A628744A25A7
:1018E20024F8E4F6D20F8007744A2524F8E4F6744B
:1018F200472524F8E66525602374452524F80674F7
:10190200452524F8E6C3940A401974472524F8A60D
:101912002574452524F8E4F6D20F80077445252462
:10192200F8E4F674582524F8E66526602374492500
:1019320024F80674492524F8E6C3940A4019745819
:101942002524F8A62674492524F8E4F6D20F800748
:1019520074492524F8E4F67D01200F024156C20F96
:10196200E5247078FC74592524F8E65D7008749DAE
:101972002CF8E4F6802874472524F8E65D70087494
:101982009D2CF87601801774582524F8E65D7008BE
:10199200749D2CF876028006749D2CF8E4F6ED25F1
:1019A200E0FD0CBC08BFE490008CF0A3F0FC9000BA
:1019B2008CE0FEA3E07802C333CE33CED8F9FF9099
:1019C200008CEEF0A3EFF0749D2CF8E6FBEE900095
:1019D2008CF0EB4FA3F00CBC08D480787C087459CF
:1019E2002524F8E65D7008749D2CF8E4F6802874CE
:1019F200472524F8E65D7008749D2CF8760180175F
:101A020074582524F8E65D7008749D2CF8760280DF
:101A120006749D2CF8E4F6ED25E0FD0CBC10BFE445
:101A220090008EF0A3F07C0890008EE0FEA3E07898
:101A320002C333CE33CED8F9FF90008EEEF0A3EF7F
:101A4200F0749D2CF8E6FBEE90008EF0EB4FA3F0C5
:101A52000CBC10D49000B3E0FF7048E524702390D2
:101A6200008CE0FAA3E0FB4A6010EB64AA7003EA80
:101A720064AA6006BA5507BB5504D2038025C20387
:101A8200802190008EE0FAA3E0FB4A6010EB64AA8A
:101A92007003EA64AA6006BA5507BB5504D20380F4
:101AA20002C203EFB4030CE4FC7C08789D7402F6D6
:031AB20008DCFC51
:011AB500220E
:1021D100E4F5247B007A007943AF24123673400280
:1021E10061777A007963AF2412367340026109AFD7
:1021F10024121FE7E52425E02415FFC007E5247517
:10220100F004A4FDACF0244AF58274003CF583E0AF
:10221100FE744B2DF58274003CF583E07C002400B4
:10222100FDEC3EFCD007E41231F9E52425E024164B
:10223100FFC007E52475F004A4FDACF0244CF58241
:1022410074003CF583E0FE744D2DF58274003CF57D
:1022510083E07C002400FDEC3EFCD007E4FB12315E
:10226100F9E52475F005A42420F582E43400F58312
:10227100E0FD7C00E52475F005A42425FFE4FB12B4
:1022810031F9E52475F005A42421F582E43400F543
:1022910083E0FD7C00E52475F005A42426FFE4FB22
:1022A1001231F9E52475F005A42422F582E4340005
:1022B100F583E0FD7C00E52475F005A42427FFE407
:1022C100FB1231F9E52475F005A42423F582E434E9
:1022D10000F583E0FD7C00E52475F005A42428FFCA
:1022E100E4FB1231F9E52475F005A42424F582E418
:1022F1003400F583E0FD7C00E52475F005A4242974
:10230100FFE4FB1231F9806EE52425E02415FFC0BE
:1023110007E52475F004A4FDACF0244AF5827400AD
:102321003CF583E0FE744B2DF58274003CF583E0AF
:102331007C002400FDEC3EFCD007E4FB1231F9E502
:102341002425E02416FFC007E52475F004A4FDACA4
:10235100F0244CF58274003CF583E0FE744D2DF5BC
:102361008274003CF583E07C002400FDEC3EFCD04F
:1023710007E4FB1231F90524E524C3940850022136
:01238100D487
:012382002238
:102A8B009000B3E070183004055356FE8003435694
:102A9B00013003055356FD8021435602801C300440
:102AAB00055356FE8003435601E544D3940040077B
:102ABB0015445356FD800343560230A008E555C319
:102ACB0013F5558008E555C3134480F55530A1081F
:102ADB00E555C313F5558008E555C3134480F555EB
:102AEB0030A208E555C313F5558008E555C31344CB
:102AFB0080F55530A308E555C313F5558008E5550A
:102B0B00C3134480F55530A408E555C313F5558020
:102B1B0008E555C3134480F55530A508E555C31397
:102B2B00F5558008E555C3134480F55530A608E5E7
:102B3B0055C313F5558008E555C3134480F555303F
:102B4B00A708E555C313F5558008E555C313448015
:102B5B00F555E4FDED75F002A42401FFE435F0FE1C
:102B6B00EF25E0FFEE33FE744A2FF58274003EF53D
:102B7B0083E0FAED75F002A42401FFE435F0FEEFDB
:102B8B0025E0FFEE33FE744B2FF58274003EF58388
:102B9B00E07E002400FFEE3AFED3EF9400EE9402A9
:102BAB004007E55713F5578008E557C3134480F5E5
:052BBB00570DBD089F4D
:012BC00022F2
:1032B1007580FF7F017E001236E778B7E624FE6055
:1032C1001A14602A24027038C2B5C2B6E5466005F8
:1032D100E4F5808003855580D2B722C2B7C2B6E536
:1032E100466005E4F5808003855680D2B522C2B7D9
:1032F100C2B5E5466005E4F5808003855780D2B606
:0133010022A9
:040FFC00759FA72214
:0436E3007F507EC3D3
:0B36E700EF1FAC0670011E4C70F622B5
:101D300000C1814001C0804101C0804100C181409B
:101D400001C0804100C1814000C1814001C080418B
:101D500001C0804100C1814000C1814001C080417B
:101D600000C1814001C0804101C0804100C181406B
:101D700001C0804100C1814000C1814001C080415B
:101D800000C1814001C0804101C0804100C181404B
:101D900000C1814001C0804101C0804100C181403B
:101DA00001C0804100C1814000C1814001C080412B
:101DB00001C0804100C1814000C1814001C080411B
:101DC00000C1814001C0804101C0804100C181400B
:101DD00000C1814001C0804101C0804100C18140FB
:101DE00001C0804100C1814000C1814001C08041EB
:101DF00000C1814001C0804101C0804100C18140DB
:101E000001C0804100C1814000C1814001C08041CA
:101E100001C0804100C1814000C1814001C08041BA
:101E200000C1814001C0804101C0804100C18140AA
:101E300000C0C101C30302C2C60607C705C5C4046A
:101E4000CC0C0DCD0FCFCE0E0ACACB0BC90908C8DA
:101E5000D81819D91BDBDA1A1EDEDF1FDD1D1CDCCA
:101E600014D4D515D71716D6D21213D311D1D0103A
:101E7000F03031F133F3F23236F6F737F53534F42A
:101E80003CFCFD3DFF3F3EFEFA3A3BFB39F9F8389A
:101E900028E8E929EB2B2AEAEE2E2FEF2DEDEC2C8A
:101EA000E42425E527E7E62622E2E323E12120E0FA
:101EB000A06061A163A3A26266A6A767A56564A4EA
:101EC0006CACAD6DAF6F6EAEAA6A6BAB69A9A8685A
:101ED00078B8B979BB7B7ABABE7E7FBF7DBDBC7C4A
:101EE000B47475B577B7B67672B2B373B17170B0BA
:101EF00050909151935352929656579755959454AA
:101F00009C5C5D9D5F9F9E5E5A9A9B5B9959589819
:101F1000884849894B8B8A4A4E8E8F4F8D4D4C8C09
:101F20004484854587474686824243834181804079
:0A3155004100490801650001630014
:10365F007E01EEA807088002C333D8FCFE1207DCF8
:04366F004E020822DD
:101FE7007E01EEA807088002C333D8FCFE6306FF14
:071FF7001207DC5E02082264
:103673007E01EEA807088002C333D8FCFE1207DCE4
:033683005E24FFC3
:013686002221
:10325700C2D8E47865F67867F6FB7A0079687F0666
:103267007EEF1227F308E6FFF46003EF70217B007F
:103277007A007968E4F5327F06123000401E7868DC
:1032870076FEE6FD7C00E4FB7F061231F9800D78BF
:1032970068E6FD7C00E4FB7F061231F97868E6FFFB
:0A32A7006003B4FF04786876FE228D
:0A36F200C2D8E47865F67867F62286
:052FFB00C213D2D82230
:03002300022E5D4D
:102E5D00C0E0C083C082C0D075D000C000C006C025
:102E6D000730987D7865E6C394325007E606246AEC
:102E7D00F8A699C298900049E0F5627865E6FF647E
:102E8D0007703A786BE6FE64036004EEB4060890B2
:102E9D0000487408F08051EEB4100B201408900017
:102EAD00487408F08042EEB4100B7870E624099057
:102EBD000048F080339000487432F0802B90004829
:102ECD00E0B5070B75620078677606D2148019EFAE
:102EDD00B40315786BE6B4190F9000487406F080B2
:102EED0007309904C299D213D007D006D000D0D0A4
:072EFD00D082D083D0E03247
:1034F400786CE6FE08E67C002400F525EC3EF52415
:10350400AF25FE1225315017754405122FFB1236D4
:10351400FCAF25AE24120B22AF25AE241213E60213
:0235240036F27D
:042531008E268F273C
:10253500900048E07865666002C322786AE6FFF499
:10254500600BEF7868666005EF6002C322786BE682
:102555006419707DFB7A00796A7D0412334A8E28EE
:102565008F29786EE6FE08E67C002400FFEC3EFE2F
:10257500EF65297003EE65286002C322786DE6FFDA
:1025850018E6FEC39F4004AD078002AD06EEC39F6B
:102595004004AF0680007868E6FEC39D4005EED393
:1025A5009F4002C322789CE6FF7E00123448123415
:1025B500117C007D1412089B8D2AE4F52BE52BC3B5
:1025C500952A500B7F647E001236E7052B80EED3EB
:1025D50022786BE6FF6403600CEF64066007EF6426
:1025E500106002C322786BE6FF64067039D3E527D5
:1025F5009408E5269400502E786DE6FEC3940250AB
:102605000990006AE030E01EC322EEC3940450092D
:1026150090006AE030E10FC322EEB4080990006A29
:10262500E030E202C322E527640A4526703CEFB498
:10263500030E1234117C007D0512089B7869A605EE
:102645007869E664016002C3221234117C007D14AE
:1026550012089B8D2AE4F52BE52BC3952A500B7F99
:10266500647E001236E7052B80EE7B007A00796ADE
:10267500900048E024FEFD12334A8E288F299000F1
:1026850048E0FD2468F8E6FE74692DF8E67C002430
:1026950000FFEC3EFEEFB52906EEB52802D322C3B6
:0126A5002212
:0413E6008E268F2799
:1013EA00E4F52CC20C786BE6FFB4061DE4F52C7408
:1013FA006A252CF8E6F599C2133013FD120FFC0585
:10140A002CE52CC3940840E722EF64036002C1561E
:10141A00786FE6F52A786AE6F52BF5991236297877
:10142A006BE6F52B3013FD123626E52A25E0F52B5F
:10143A003013FD123626E52CC3952A4002C1397EA7
:10144A0000E527252CFFEE3526FEC3EF9464EE94C3
:10145A00005060E52C2527FF7B007A007928E4F507
:10146A0031121F304005E4F528F5297E00E52725CD
:10147A002CFFEE3526FEC3EF944EEE94004005E4B1
:10148A00F52B8004E528F52B3013FD1236267E0055
:10149A00E527252CFFEE3526FEC3EF944EEE940089
:1014AA004005752B018004E529F52B3013FD123612
:1014BA0026C1357E00E527252CFFEE3526FEEF6492
:1014CA00634E7016F52B3013FD12362690006AE033
:1014DA00F52B3013FD123626C135AF2C7E00E527D9
:1014EA00252CCFEE3526CF249CCF34FFFEC3EF94B4
:1014FA0012EE9400504E7E00E527252CFFEE35268D
:10150A00FEEF25E0FFEE33FE74A42FF58274FF3E52
:10151A00F583E0F52B3013FD1236267E00E52725EC
:10152A002CFFEE3526FEEF25E0FFEE33FE74A42FE6
:10153A00F58274FF3EF583E0A3E0F52B3013FD122C
:10154A003626C1357E00E527252CFFEE3526FEC35B
:10155A00EF9486EE94005051EF248AFFEE34FFFE9A
:10156A00EF25E0FFEE33FE744A2FF58274003EF554
:10157A0083E0F52B3013FD123626AF2C7E00E527CB
:10158A00252CCFEE3526CF248ACF34FFFEEF25E077
:10159A00FFEE33FE744B2FF58274003EF583E0F5BF
:1015AA002B3013FD123626C1357E00E527252CFF88
:1015BA00EE3526FED3EF94ADEE94005021E4F52BE0
:1015CA003013FD123626E52C2527249AF582E434B9
:1015DA00FFF583E0F52B3013FD123626804D7E0091
:1015EA00E527252CFFEE3526FEEF64AE4E702AF570
:1015FA002B3013FD1236267B007A007928E4F53168
:10160A007F4D121F3040067528007529FFE529F520
:10161A002B3013FD1236268012E4F52B3013FD12FF
:10162A003626752B013013FD123626052C8140C251
:10163A000C3013FD7864E6F599C2133013FD786611
:10164A00E6F599C213301302C1EE80F9786BE664AD
:10165A00107038F52C746A252CF8E6F52BF599C22A
:10166A00133013FDAF2B12362D120FFC052CE52C6F
:10167A00C3940640E07864E6F599C2133013FD7806
:10168A0066E6F599C21320135B80FB786BE6641952
:10169A00705218E6F52BF599C2133013FDAF2B12D1
:1016AA00362D120FFC786BE6F52BF599C213301321
:1016BA00FDAF2B12362D120FFC7868E6F52BF59943
:1016CA00C2133013FDAF2B12362D120FFC7864E6CD
:1016DA00F599C2133013FD7866E6F599C2133013F3
:0416EA00FD120FFCE2
:0116EE0022D9
:040B22008E268F2765
:100B2600752C01E4F52D786BE664066002C184C37A
:100B3600E5279464E52694004002A129786DE694A1
:100B460001502C786FE6FD7C00E4FBFF1231F9784A
:100B56006EE6FD7C00E4FB7F011231F990006AE04D
:100B66004401F0FD7C00E4FB7F631231F9C1FB78A0
:100B76006DE6D39403502D786FE6FD7C00E4FB7F91
:100B8600021231F9786EE6FD7C00E4FB7F03123138
:100B9600F990006AE04402F0FD7C00E4FB7F6312FA
:100BA60031F9C1FB786DE66408702E08E6FE08E6AA
:100BB6007C002400FDEC3EFCE4FB7F081231F9903A
:100BC600006AE04404F0FD7C00E4FB7F631231F927
:100BD600786FE690006BF0C1FB786DE6B4091B08F0
:100BE600E6FE08E67C002400FDEC3EFCE4FB7F0903
:100BF6001231F9786FE6F51CC1FB786DE6FFB40695
:100C06001C786FE6FD7C00E4FB1231F9786FE6781C
:100C160068F67D067CEFE4FF123561C1FB786DE670
:100C2600FFB40D1FC00708E6FE08E67C002400FDA1
:100C3600EC3EFCD007E4FB1231F9786FE69000B188
:100C4600F0C1FB786DE6FFB40C1B786FE6FD7C0007
:100C5600E4FB1231F9786FE69000B3F06002C1FB55
:100C6600754601C1FB786DE6FFB41012786FE6FD9C
:100C76007C00E4FB1231F9786FE6F52CC1FB786D48
:100C8600E6640A70277869E664016002C1FB786F42
:100C9600E6FD7C00E4FB7F061231F9786FE67868A2
:100CA600F67D067CEFE4FF123561C1FBE527640F94
:100CB6004526702B786DE6FF786FE6FD7C00E4FB39
:100CC6001231F9786FE6B4010B758780900049748C
:100CD60003F0C1FBE4F5879000497406F0C1FBE51B
:100CE6002764144526702B786DE6FF786FE6FD7C49
:100CF60000E4FB1231F9786FE6B4010B758780903A
:100D060000497403F0C1FBE4F5879000497406F0CE
:100D1600C1FB786DE6FF786FE6FD7C00E4FB1231DF
:100D2600F9C1FBC3E527942CE52694014002C1FBDB
:100D3600786CE67F00FE08E67C002400FFEC3ECFE0
:100D4600249CF527EF34FFF526D3E5279412E526F4
:100D56009400503808E6FE08E62400F529EC3EF536
:100D660028D3E52994FFE528648094834002C1FBDB
:100D7600E52725E0FFE52633FE746C2FF582740027
:100D86003EF583E528F0A3E529F0C1FBD3E52794DA
:100D960049E52694004002C137C3E5279422E5269B
:100DA60094005002C1FBE52724DEFFE52634FFFE52
:100DB6007C007D051208468F2B7B007A0079431252
:100DC60036734002C1FBE52724DEFFE52634FFFE2D
:100DD6007C007D05120846ED4C70437A007963AFBE
:100DE6002B12365FE52B25E025E02400F582E4345E
:100DF60000F583120AF100000000E52B25E025E04E
:100E060024B8F582E43400F583120AF100000000EC
:100E1600AF2B12357F7DF47C017F0812348C786FFE
:100E2600E6FF74FE2527F582E434FFF583EFF0C173
:100E3600FBE527644A4526701F786FE6F543F52BD8
:100E4600FF1235A3E52BFD7C00E4FB7F4D1231F943
:100E56009000B6741EF0C1FBE52764634526600268
:100E6600C1FB786FE6752800F529E4FBAD29AC28AF
:100E76007F631231F9786FE690006AF08077786BBD
:100E8600E664107070786FE6F9786CE6FE08E67C2A
:100E9600002400F527EC3EF526749C2527F52774DB
:100EA600FF3526F526E4FDE9FFC3ED9FEC940050DF
:100EB60044120FFCAF05EF25E0FB2471F8E6FE7443
:100EC600722BF8E67A002400F529EA3EF528E52794
:100ED6002DFFE5263CFEEF25E0FFEE33FE746C2F7A
:100EE600F58274003EF583E528F0A3E529F00DBDF3
:100EF60000010C80B2E52C647F70357F7712364393
:100F0600E4F52A7B007A00792BE4F532AF2A123019
:100F160000500DE4252AFDE434EEFCAF2B123561BA
:100F2600052AE52AD3941040DAC2AF759F8080FE69
:0C0F3600E52CB4FF07C2AF759F8080FE61
:010F4200228C
:0936FC00786676FF786476FF22FF
:07362600852B99C213AF2BA5
:10362D007864E66FFF901D30937866667964F7EFE6
:05363D00901E3093F621
:013642002265
:08334A008B2C8A2D892E8D2F9A
:103352007530007531FF7DFFAF2F152FEF6026AB63
:103362002C052EE52EAA2D7002052D14F91207DC6C
:103372006531FF901D30936D753000F531EF901E71
:0A3382003093FD80D3E531FEEDFF2E
:01338C00221E
:02368700000041
:07315F004100B708011C004C
:10345200E4F524751C01D20C7F08122CCE500375A2
:103462002401751C02120F435003752402751C03BC
:1034720012338DEFD3940040028F2485241CE51C67
:0A348200FD7C00E4FB7F090231F934
:100F430012318E9000B7E0FF139290EFA2E19291DD
:100F5300A2E292927FB11235C712308EEF4E600536
:100F6300123705C3227F017E001236E71233028E49
:100F73001A8F1B1235264005123705C3227F017EC7
:100F8300001236E71233028E258F261235264005CE
:100F9300123705C3227F017E001236E71233028E19
:100FA300278F28123705E51B2526FFE51A3525541B
:100FB30003F5298F2A9000B7E0B40815E528B52A70
:100FC30027E527B529227D0FAF26AE2512294A80B2
:100FD30017E528B52A12E527B5290D9000B7E014C7
:100FE300FDAF26AE2512294A9000B7E004F0E0D306
:080FF300940F40037408F0D3D1
:010FFB0022D3
:10357F008F2E12318E7FB81235C712308EEF4E60FC
:10358F00030237057F017E001236E7AF2E1235C7D3
:04359F0012370522B8
:10338D0012318E7FB91235C712308EEF4E60061294
:10339D0037057F00227F017E001236E71233028F40
:1033AD00251235267F017E001236E71233028F2655
:1033BD00E5256226123705E52670028003E4F52522
:0233CD00AF252A
:0133CF0022DB
:1035A3008F2E12318E7FBA1235C712308EEF4E60D6
:1035B300030237057F017E001236E7AF2E1235C7AF
:0435C3001237052294
:102DAD0012318E7FB71235C712308EEF4E6003028F
:102DBD0037057F017E001236E79000B7E024F8FF5B
:102DCD001235C712308EEF4E60030237057F017E3C
:102DDD00001236E71233028F161235267F017E0060
:102DED001236E78516251233028F171235267F010D
:102DFD007E001236E7E51762251233028F18123561
:102E0D00267F017E001236E7E51862251233028F08
:102E1D00191235267F017E001236E7E5196225125B
:102E2D0033028F1DE51D6225123705E5257011AFA3
:102E3D0019AE18AD17AC169000B7E0F52A1226A6FC
:0F2E4D009000B7E004F0E0D3940F40037408F056
:012E5C002253
:022CCE008F2550
:102CD00078267C007D007BFF7A3679877E007F1422
:102CE0001207B6C290C291C29212318E300C077F89
:102CF000B11235C78008200C057FB21235C77F019D
:102D00007E001236E712308EEF4E6005123705C393
:102D1000227F017E001236E71233028E268F27753E
:102D20003A011235264005123705C3227F017E0085
:102D30001236E7E53A139290E53AA2E19291A2E2C7
:102D40009292123302E53A25E02426F8A60608A658
:102D500007053AE53AD3940940C8123705E5272517
:102D600029CFE5263528CF252BCF352ACF252DCFC6
:102D7000352CCF252FCF352ECF2531CF3530CF2550
:102D800033CF3532CF2535CF3534CF2537CF353614
:102D90005403FEE539B50713E538B5060E7B007A16
:0C2DA00000792685253F7D08122383D38F
:012DAC002204
:10318E00C2967F017E001236E7D297D2967F027EDC
:10319E00001236E7C2977F057E001236E7C2967F91
:1031AE00027E001236E7E51CB4021DD297D2967F3E
:1031BE00027E001236E7C2977F057E001236E7C206
:1031CE00967F027E000236E7E51CB4031DD297D22D
:1031DE00967F027E001236E7C2977F057E0012367A
:0B31EE00E7C2967F027E001236E72247
:10352600E4FFFE20970D0FBF00010EEF64644E709E
:10353600F2C322D2977F017E001236E7D296C29757
:0C3546007F017E001236E7D297C296D3B8
:013552002256
:0235C700AD074E
:1035C9007B08ED339297D2967F017E001236E7C2CF
:0E35D900967F017E001236E7ED25E0FDDBE473
:0135E70022C1
:10330200E4F53BF53CE51CB403047A0880027A0A32
:10331200E4FBEBC39A502CD2967F017E001236E773
:10332200D297E53C25E0FFE53B33FEA297E433FD6F
:10333200EEF53BEF4DF53CC2967F017E001236E77B
:073342000B80CFAE3BAF3C56
:013349002261
:07370500C297D296D2972271
:10308E00E4F53BF53CE51C64017022D297D296FA2A
:10309E00FB209707C2967E007F00220BBB00010A21
:1030AE00EB640A4A70EBC2967E007F0122E51C6437
:1030BE00027027FAFB209710D2967F017E001236FF
:1030CE00E7C2967E007F00220BBB00010AEB643242
:1030DE004A70E2C2967E007F0122E51C64037028CE
:1030EE00FAFBD297209710D2967F017E001236E718
:1030FE00C2967E007F00220BBB00010AEB64324AAF
:08310E0070E0C2967E007F0113
:013116002296
:06294A008E2B8F2C8D2D59
:10295000E52D25E0246CF582E43400F583E0FEA348
:10296000E0FFC3E52C9FFFE52B9EFE1236D1D3EF8F
:102970009464EE64809480403B74D8252DF582E405
:102980003400F583E004F074D8252DF582E434009A
:10299000F583E0D3648094825002412CE4F0E52D6D
:1029A00025E0246CF582E43400F583E52BF0A3E503
:1029B0002CF0807874D8252DF582E43400F583E47A
:1029C000F0E52D25E0246CF582E43400F583E0FE8B
:1029D000A3E0FFE4FCFD7B02FAF9F81209A1C004B0
:1029E000C005C006C007AE2BAF2CE4FCFD7B08FA87
:1029F000F9F81209A1D003D002D001D000EB2FFFCB
:102A0000EA3EFEE93DFDE83CFCE47B0AFAF9F812F7
:102A10000A2C8F318E308D2F8C2EE52D25E0246CE5
:102A2000F582E43400F583EEF0A3EFF0E52D25E028
:102A3000246CF582E43400F583E0FEA3E0D3940037
:102A4000EE94044013E52D25E0246CF582E4340077
:102A5000F5837404F0A3E4F0E52D25E0246CF58201
:102A6000E43400F583E0FEA3E0FFE4FCFD7B607A44
:102A7000EAF9F8C3120ABE5011E52D25E0246CF5E1
:0A2A800082E43400F583E4F0A3F0D3
:012A8A002229
:0826A6008F298E288D278C2658
:1026AE00E52A24F8F52B7B007A007943FF12367366
:1026BE004002E1B89000B6E06062E52A25E025E030
:1026CE0024E0F582E434FFF583E0FCA3E0FDA3E013
:1026DE00FEA3E02529FFEE3528FEED3527FDEC356E
:1026EE0026FCE52B25E025E0244AF582E43400F5AE
:1026FE0083120AE5AF29AE28AD27AC26E52B25E0DF
:10270E0025E024B8F582E43400F583120AE5E543AA
:10271E00F46002E1F29000B6E014F022E52B25E021
:10272E0025E024B8F582E43400F583E0F8A3E0F95F
:10273E00A3E0FAA3E0FBC3E5299BFFE5289AFEE59B
:10274E002799FDE52698FCE47BFF7AFFF9F8D31272
:10275E000AD45002E1F2E52A25E025E024E0F582D4
:10276E00E434FFF583E0FCA3E0FDA3E0FEA3E02547
:10277E0029FFEE3528FEED3527FDEC3526FCE52B41
:10278E0025E025E0244AF582E43400F583120AE5BB
:10279E00AF29AE28AD27AC26E52B25E025E024B8E1
:1027AE00F582E43400F583020AE5E47FFF7E03FD43
:1027BE00FCAB29AA28A927A826D3120AD4400BE4D9
:1027CE007529FF752803F527F526AF29AE28AD2705
:1027DE00AC26E52B25E025E0244AF582E43400F50D
:0427EE0083120AE563
:0127F20022C4
:082383008B3B8A3C893D8D3E35
:10238B00E4F542E542C3953E4002A130AB3BAA3C8B
:10239B00A93DE5420475F002A4F58285F08312098C
:1023AB0012FFAEF0E542253F25E0246CF582E434C4
:1023BB0000F583E0FCA3E0FDC3EF9DF541EE9CF53A
:1023CB0040C3E5419464E54064809480500DC3E5BF
:1023DB0041949CE5406480947F5023E542253FFD6A
:1023EB0025E0246CF582E43400F583EEF0A3EFF0E6
:1023FB0074D82DF582E43400F583E4F08058E5427F
:10240B00253FF925E0246CF582E43400F583E0FCEC
:10241B00A3E0FDC39FEC9E500F74D829F582E434E2
:10242B0000F583E004F0802EAB3BAA3CA93DE542CE
:10243B000475F002A4F58285F083120912FFD3ED27
:10244B009FEC95F04010E542253F24D8F582E4340B
:10245B0000F583E014F0E542253FFB24D8F582E438
:10246B003400F583E0FFD36480948A500AC3EF6491
:10247B008094764002A12CD3E5419414E54064800E
:10248B009480500DC3E54194ECE5406480947F50FB
:10249B001FAE40AF417C007D0512089BEB25E0246D
:1024AB006CF582E43400F583EE8FF01208D1806274
:1024BB00AB3BAA3CA93DE5420475F002A4F582852D
:1024CB00F083120912FFAEF0E542253FFD25E02413
:1024DB006CF582E43400F583E0FAA3E0FBC39FEADA
:1024EB009E5015ED25E0246CF582E43400F583E471
:1024FB0075F0011208D1801AD3EB9FEA9E4013EDC1
:10250B0025E0246CF582E43400F58374FFF5F012BA
:10251B0008D1E542253F24D8F582E43400F583E465
:05252B00F00542618E85
:012530002288
:1034C1000205050506060606070707080809090A91
:1034D1000B0C0C0D0E10121315171B1E252A2F365F
:1034E1003A3B37312C26231E1D18181515131111BF
:0334F100100F0FAA
:0E31660041011200011E00C115420113012C8F
:10028C00E4F526F527200A3BD293A29033FDA291E8
:10029C00E433FBA292E433FAE51F139290E51FA21C
:1002AC00E19291A2E29292C2B37FF47E011236E700
:1002BC00D2B3ED24FF9290EB24FF9291EA24FF92AB
:1002CC0092C293E51F045407F51F9000B3E0F96048
:1002DC000261E0300A6C20020261E0900112E064DD
:1002EC000C7057E51E045407F51EC202D2083015D7
:1002FC002625E0246CF582E43400F5837403F0A326
:10030C0074E8F0E51EB40702C215E4900112F0E5A2
:10031C0046602715468023E51E25E0246CF582E413
:10032C003400F583E4F0A3F0E51EB40702D215E423
:10033C00900112F0E54660021546900112E004F0BF
:10034C0061E020020261E0E51F30E015900113E04E
:10035C00FEA3E0FFC374E89FF52574039EF524808B
:10036C000A900113E0F524A3E0F525C37407951F4B
:10037C0025E0246CF582E43400F583E524F0A3E554
:10038C0025F0900112E064207044C202D2083015AE
:10039C001B900114E02464F0900113E03400F0E0B1
:1003AC00B40320A3E0B4E81BC2158017900114E03D
:1003BC00249CF0900113E034FFF0E07002A3E07095
:1003CC0002D215E4900112F0E54660021546900148
:1003DC0012E004F0200A02C184E51FB408004002B8
:1003EC00C1E59003F425E0738104815481A481F468
:1003FC00A144A194A1E4C134749D251FF8E6FF70BB
:10040C000CE96009300003C2A022D2A022EFB40193
:10041C000CE96009300003D2A022C2A022E51F25FE
:10042C00E0246CF582E43400F583E0FEA3E0D39481
:10043C00F4EE94014009300003D2A022C2A0223075
:10044C000003C2A022D2A022749D251FF8E6FF70E3
:10045C000CE96009300003C2A122D2A122EFB40141
:10046C000CE96009300003D2A122C2A122E51F25AC
:10047C00E0246CF582E43400F583E0FEA3E0D39431
:10048C00F4EE94014009300003D2A122C2A1223023
:10049C000003C2A122D2A122749D251FF8E6FF7091
:1004AC000CE96009300003C2A222D2A222EFB401EF
:1004BC000CE96009300003D2A222C2A222E51F255A
:1004CC00E0246CF582E43400F583E0FEA3E0D394E1
:1004DC00F4EE94014009300003D2A222C2A22230D1
:1004EC000003C2A222D2A222749D251FF8E6FF703F
:1004FC000CE96009300003C2A322D2A322EFB4019D
:10050C000CE96009300003D2A322C2A322E51F2507
:10051C00E0246CF582E43400F583E0FEA3E0D39490
:10052C00F4EE94014009300003D2A322C2A322307E
:10053C000003C2A322D2A322749D251FF8E6FF70EC
:10054C000CE96009300003C2A422D2A422EFB4014A
:10055C000CE96009300003D2A422C2A422E51F25B5
:10056C00E0246CF582E43400F583E0FEA3E0D39440
:10057C00F4EE94014009300003D2A422C2A422302C
:10058C000003C2A422D2A422749D251FF8E6FF709A
:10059C000CE96009300003C2A522D2A522EFB401F8
:1005AC000CE96009300003D2A522C2A522E51F2563
:1005BC00E0246CF582E43400F583E0FEA3E0D394F0
:1005CC00F4EE94014009300003D2A522C2A52230DA
:1005DC000003C2A522D2A522749D251FF8E6FF7048
:1005EC000CE96009300003C2A622D2A622EFB401A6
:1005FC000CE96009300003D2A622C2A622E51F2511
:10060C00E0246CF582E43400F583E0FEA3E0D3949F
:10061C00F4EE94014009300003D2A622C2A6223087
:10062C000003C2A622D2A622749D251FF8E6FF70F5
:10063C000CE96009300003C2A722D2A722EFB40153
:10064C000CE96009300003D2A722C2A722E51F25BE
:10065C00E0246CF582E43400F583E0FEA3E0D3944F
:10066C00F4EE94014009300003D2A722C2A7223035
:10067C000003C2A722D2A722C37407951F249DF89A
:10068C00E6FF700A9000B3E06004E4F5A722EFB433
:10069C0001109000B3E0600A7FFF7E03122F048FDD
:1006AC00A722C37407951F25E0246CF582E434005F
:1006BC00F583E0FEA3E0FF9000B1E0FD7C00EF2DA0
:1006CC00FFEC3ECF2480CF34FFFEC3648094805077
:0906DC0003E4FEFF122F048FA7B6
:0106E50022F2
:042F04008E288F295B
:102F0800E4F52A9034C193752B00F52CD3E52C9564
:102F180029E52B95284006E4FAFBFFFE22052AAF97
:102F28002AEF3395E0FE74C12FF58274343EF583A1
:102F3800E493F9252CF52CE4352BF52BD3E52C95CA
:102F480029E52B95284050E52C9529FFE52B952858
:102F5800FEE9C39FFBE49EFA7C007D0AAF03FE12E4
:102F68000834AA06AB07E9FD12089BAA06AB077C42
:102F7800007D051208347D0A12089BAA06AB07AF2C
:102F88002AEF3395E0FE7C007D05120834EF2BFB19
:102F9800EE3AFAAF03FE22E52A7082FA7BFF7FFF42
:012FA800FE2A
:012FA9002205
:03010000140012D6
:10317400440104020002004800FC00680069006683
:0931840000674400F8000200029B
:0E355300853583E493FF90010FF0AC37AD385F
:10356100AB07C2AF75F65575F6AA75F65543BF049C
:0E3571008CF48DF58BF675F780D2AF7F0022BB
:10364300C2AF75F65575F6AA75F65543BF04EF2557
:0C365300E0F5F4E4F5F575F782D2AF2243
:0B27F3008F828E83E4931208227F0186
:0127FE0022B8
:0C35E800E52575F002A4240CF9E4FAFBC0
:1035F4001208E7F58285F083E4932402FFE4338F15
:04360400F002094A7D
:0233D000A9074B
:1033D200E925E024F8F582E43400F583E0A3E0F582
:1033E20034E925E0240CF8E6FE08E6FFE534240281
:1033F200FDE433FCE925E02410F8E6FA08E6C39D73
:0E340200FDEA9CFCC3EF9DEE9C4002D322C36A
:013410002299
:1036BF00E4F524AF24121AB60524E524C39402407E
:0136CF00F208
:0136D00022D7
:021AB6008F257A
:101AB800EF25E02404F582E43401F583E0F528A35A
:101AC800E0F529EF25E025E024FCF582E43400F573
:101AD80083E0A3E0F526EF25E025E024FEF582E487
:101AE8003400F583E0A3E0F527E52625E0F52A751F
:101AF8002B00E52725E0752CFFF52D752E00852B8D
:101B080082852A83E49364556002815EAB2CAA2DFA
:101B1800A92E1207DC64556002815EE52B2401FFC3
:101B2800E4352AFEE52525E0240CF8A60608A607D4
:101B3800E52525E0240CF8E6FE08E6F5828E83E428
:101B480093F46020E52525E0240CF8E6FE08E6AAD3
:101B580006C3852D83852E829582EA9583500512CA
:101B680035E880CCE52525E0240CF8E6FE08E6C338
:101B7800952BF530EE952AF52FE52E2401F9E4355D
:101B88002DFEAF01E52525E0240CF8A60608A607DA
:101B9800E52525E0240CF8E6FE08E6F5828E83E4C8
:101BA80093F46030AB2CE52E2529F9E52D3528FA7C
:101BB800C0038A838982E52525E0240CF8E6FE081F
:101BC800E6AA06F9C3D0E0E99582EA9583500512A2
:101BD80035E880BCE52525E0240CF8E6FE08E6ABF0
:101BE8002CAA2DA92EAC02AD01C39DFFEE9CFED3FD
:101BF800EF9530EE952F5032AE02AF01EF2401FF82
:101C0800E43EFEE52525E02408F8A60608A60774A4
:101C1800142525F8A626AE2AAF2BAD07AC06E4FF9F
:101C2800123561EF700281DFC322E52B2401FFE446
:101C3800352AFEE52525E02408F8A60608A6077437
:101C4800142525F8A627AC2DAD2EE4FF123561EF3B
:101C5800700281DFC322852B82852A83E493B455E1
:101C68001EE52B2401FFE4352AFEE52525E024089E
:101C7800F8A60608A60774142525F8A6278058ABE9
:101C88002CAA2DA92E1207DCB45520AE02AF01EF05
:101C98002401FFE43EFEE52525E02408F8A6060811
:101CA800A60774142525F8A626802CAE2AAF2BADDE
:101CB80007AC06ED2401FFE43CFEE52525E02408F9
:101CC800F8A60608A60774142525F8A6277F551236
:101CD8003561EF6002C322E52525E02408F8E6FE19
:101CE80008E6FFE52525E0240CF8A60608A607E582
:101CF8002525E02408F8E6FE08E62529FFE5283E24
:101D0800FEE52525E02410F8A60608A607E5252502
:101D1800E0240CF8E6FE08E6F5828E83E493F4608E
:071D2800051235E880E7D346
:011D2F002291
:022000008F341B
:10200200EF25E02408F8E6FE08E68E35F53674146E
:102012002FF8E625E0F537753800E53425E024048D
:10202200F582E43401F583E0FFA3E0900110CFF0E4
:10203200A3EFF0E490010CF0E53425E02404F582EE
:10204200E43401F583E0C313FF90010CE0C39FE485
:1020520094005015120FFC74142534F8E6FFE02F9B
:10206200FF123643E004F080CFAF36900111E02535
:1020720036FF900110E03535CF24FFF53AEF34FFFB
:10208200F5390538E538700205378536828535839E
:10209200E493F470022133C3E536953AE535953978
:1020A20040022133120FFC853682853583740193F9
:1020B200FF6073F46070E493FF90010D12355CEFE2
:1020C20060037F01220538E538700205370536E5E1
:1020D2003670020535F582123553EF60037F012217
:1020E2000538E538700205370536E53670020535E4
:1020F200E490010CF090010DE0FF90010CE0C39F11
:102102005088853682123553EF60037F01220538ED
:10211200E538700205370536E5367002053590015F
:102122000CE004F080CF7B007A0079351235F4019F
:102132008CE53425E0240CF8A63708A638E53425CA
:10214200E02408F8E6FE08E6EEC313FF90010EF065
:10215200FD74142534F8E625E0FEE53425E0240874
:10216200F8A60608760074142534F8A605E5342589
:10217200E02408F8E6FE08E6FF900111E02FFF9048
:102182000110E03EFEE53425E02410F8A60608A67C
:1021920007E53425E02408F8E6FC08E6FD7F551241
:1021A2003561EF60037F012274142534F8E67D0067
:1021B20025E0FCE4FF123561EF60037F0122E53484
:0E21C20025E02408F80806E6700218067F00E3
:0121D00022EC
:082800008F348B358A368937CD
:10280800E4F53DF53EE53825E024F8F582E43400AA
:10281800F583E0A3E0F53FE53825E02408F8E6FE77
:1028280008E68E39F53A0534E53825E0240CF8E653
:10283800FE08E6FFE53F2401FDE433FCE53825E02A
:102848002410F8E6FA08E6C39DFDEA9CFCD3EF9D48
:10285800EE9C400122853A82853983740193FE6596
:10286800346010E493F4600B7B007A0079391235F8
:10287800F480E2EEB5340BE53A2401F53EE435394F
:10288800F53DE53825E0240CF8E6FE08E6FFFDAC4A
:1028980006AF3F1235618F3BE53B6002C322E53846
:1028A80025E0240CF808740226F618E436F6E4F558
:1028B8003CE53CC3953F5033E53825E0240CF8E669
:1028C800FE08E6253CFFE43EFEAD07FCAB35AA3624
:1028D800A937853C827583001207F5FF1235618F91
:1028E8003BE53B6002C322053C80C6AF3F7E00E566
:1028F8003825E0240CF808EF26F618EE36F6E53809
:1029080025E0240CF8E6FC08E6FDEF2401FFEE3391
:10291800FEC3ED9FFFEC9EFEAD07FCAF34123561A0
:102928008F3BE53B6002C322E53E453D6012AE3D6C
:10293800AF3EAD07AC06E4FF123561EF6002C3227B
:01294800D3BB
:01294900226B
:081F30008F2D8B2E8A2F8930C2
:101F3800E53125E02408F8E6FE08E68E32F533E4BC
:101F4800F534F535052D853382853283E493F460C5
:101F580049E53125E02410F8E6FC08E6FDC3E53341
:101F68009DE5329C5034740193652D7022E535450A
:101F7800346016E5352401FFE43534FEAD07FCE492
:101F8800FF123561EF6002C3228532348533357B19
:101F9800007A0079321235F480ACE5354534603D7D
:101FA800853582853483740293FFAB2EAA2FA9301E
:101FB800E48FF0120982AB2EAA2FA9301208E77518
:101FC800F000120982853582853483740393FFAB50
:0E1FD8002EAA2FA930E48FF012094AD322C39B
:011FE60022D8
:083000008F2E8B2F8A308931DD
:10300800E53225E02408F8E6FE08E68E33F534E4D8
:10301800F535F536052E853482853383E493F460DF
:1030280049E53225E02410F8E6FC08E6FDC3E5345E
:103038009DE5339C5034740193652E7022E5364526
:10304800356016E5362401FFE43535FEAD07FCE4AE
:10305800FF123561EF6002C3228533358534367B34
:10306800007A0079331235F480ACE53645356014C2
:10307800853682853583740393AB2FAA30A9311224
:053088000822D322C361
:01308D002220
:0431F9008F2E8B2F5B
:1031FD00E4F530EDF532ECF531120FFCAF2F123353
:10320D00D05022E530C3940A500CAF2F122000EF9E
:10321D006004053080ED7F057E001236E7E530C392
:10322D00940A400122E530C3940A50147B007A00C1
:10323D007931852F38AF2E1228004004053080E5F6
:09324D00E530C3940A400122D3CC
:013256002255
:03000000020200F9
:0C020000787FE4F6D8FD7581B702024754
:1006E600E709F608DFFA8046E709F208DFFA803EF6
:1006F60088828C83E709F0A3DFFA8032E309F608E3
:10070600DFFA8078E309F208DFFA807088828C834A
:10071600E309F0A3DFFA806489828A83E0A3F608FE
:10072600DFFA805889828A83E0A3F208DFFA804CD8
:1007360080D280FA80C680D4806980F280338010AF
:1007460080A680EA809A80A880DA80E280CA803318
:1007560089828A83ECFAE493A3C8C582C8CCC58390
:10076600CCF0A3C8C582C8CCC583CCDFE9DEE78060
:100776000D89828A83E493A3F608DFF9ECFAA9F0DF
:10078600EDFB2289828A83ECFAE0A3C8C582C8CC35
:10079600C583CCF0A3C8C582C8CCC583CCDFEADE4E
:1007A600E880DB89828A83E493A3F208DFF980CCB0
:1007B60088F0EF60010E4E60C388F0ED2402B404A9
:1007C6000050B9F582EB2402B4040050AF23234550
:0607D60082239007367338
:1007DC00BB010689828A83E0225002E722BBFE021B
:0907EC00E32289828A83E493224E
:1007F500BB010CE58229F582E5833AF583E02250B9
:1008050006E92582F8E622BBFE06E92582F8E22202
:0D081500E58229F582E5833AF583E493221C
:10082200BB010689828A83F0225002F722BBFE01B5
:02083200F322AF
:10083400EF8DF0A4A8F0CF8CF0A428CE8DF0A42ED8
:02084400FE2292
:10084600BC000BBE0029EF8DF084FFADF022E4CC96
:10085600F875F008EF2FFFEE33FEEC33FCEE9DEC5F
:10086600984005FCEE9DFE0FD5F0E9E4CEFD22EDA5
:10087600F8F5F0EE8420D21CFEADF075F008EF2FEF
:10088600FFED33FD4007985006D5F0F222C398FDE0
:050896000FD5F0EA227D
:10089B00C2D5EC30E709B2D5E4C39DFDE49CFCEE78
:1008AB0030E715B2D5E4C39FFFE49EFE120846C3A2
:1008BB00E49DFDE49CFC800312084630D507C3E49D
:0608CB009FFFE49EFE22E7
:1008D100C5F0F8A3E028F0C5F0F8E58215827002B2
:0608E1001583E038F0224F
:1008E700BB010A89828A83E0F5F0A3E022500687DC
:1008F700F009E71922BBFE07E3F5F009E31922899E
:0B090700828A83E493F5F074019322D0
:10091200BB0110E58229F582E5833AF583E0F5F023
:10092200A3E0225009E92582F886F008E622BBFE00
:100932000AE92582F8E2F5F008E222E5832AF58346
:08094200E993F5F0A3E993220B
:10094A00BB010789828A830208D1500B09C5F027A7
:10095A00F7C5F01937F722BBFE0D09F8E325F0F3C6
:10096A00C5F019E338F322F889828A837401932542
:08097A00F0C5F0F8E493382207
:10098200BB010A89828A83F0E5F0A3F0225006F7C0
:0F09920009A7F01922BBFE06F3E5F009F31922BD
:1009A100E88FF0A4CC8BF0A42CFCE98EF0A42CFCF5
:1009B1008AF0EDA42CFCEA8EF0A4CDA8F08BF0A473
:1009C1002DCC3825F0FDE98FF0A42CCD35F0FCEBD2
:1009D1008EF0A4FEA9F0EB8FF0A4CFC5F02ECD3997
:0F09E100FEE43CFCEAA42DCE35F0FDE43CFC2204
:1009F00075F008758200EF2FFFEE33FECD33CDCCBE
:100A000033CCC58233C5829BED9AEC99E582984040
:100A10000CF582EE9BFEED9AFDEC99FC0FD5F0D61D
:100A2000E4CEFBE4CDFAE4CCF9A88222B800C1B947
:100A30000059BA002DEC8BF084CFCECDFCE5F0CB85
:100A4000F97818EF2FFFEE33FEED33FDEC33FCEBBE
:100A500033FB10D703994004EB99FB0FD8E5E4F979
:100A6000FA227818EF2FFFEE33FEED33FDEC33FC66
:100A7000C933C910D7059BE99A4007EC9BFCE99A5A
:100A8000F90FD8E0E4C9FAE4CCFB2275F010EF2F9F
:100A9000FFEE33FEED33FDCC33CCC833C810D7079F
:100AA0009BEC9AE899400AED9BFDEC9AFCE899F8DA
:0E0AB0000FD5F0DAE4CDFBE4CCFAE4C8F9226D
:100ABE00EB9FF5F0EA9E42F0E99D42F0EC6480C8AF
:060ACE0064809845F0224F
:100AD400EB9FF5F0EA9E42F0E99D42F0E89C45F078
:010AE40022EF
:0C0AE500ECF0A3EDF0A3EEF0A3EFF02284
:100AF100A8828583F0D083D082120B08120B0812D2
:100B01000B08120B08E473E493A3C583C5F0C583F6
:100B1100C8C582C8F0A3C583C5F0C583C8C582C84E
:010B210022B1
:10341100AC5DAD5EAE5FAF60780FEFA2E2EC20E68F
:1034210001B35D5E5FF47004FCFDFEFFEF13FFEE80
:1034310013FEED13FDEC13FCD8E08C5D8D5E8E5F09
:103441008F60EE547FFE228E5D8F5EE4F55FF56046
:013451002258
:1036D100C3EE6480948040028007C3E49FFFE49EB0
:0236E100FE22C7
:10020C000216EFE493A3F8E493A34003F68001F203
:10021C0008DFF48029E493A3F85407240CC8C333F3
:10022C00C4540F4420C8834004F456800146F6DFC2
:10023C00E4800B0102040810204080903117E47E0A
:10024C00019360BCA3FF543F30E509541FFEE493B7
:10025C00A360010ECF54C025E060A840B8E493A37E
:10026C00FAE493A3F8E493A3C8C582C8CAC583CAA9
:10027C00F0A3C8C582C8CAC583CADFE9DEE780BE61
:01318D000041
:00000001FF
